:020000040800F2
:10000000B036002019010008210100082301000872
:100010002501000827010008290100080000000050
:100020000000000000000000000000002B0100089C
:100030002D010008000000002F010008B102000897
:1000400033010008330100083301000833010008C0
:1000500033010008330100083301000833010008B0
:1000600033010008330100083301000833010008A0
:100070003301000833010008330100083301000890
:100080003301000833010008330100083301000880
:1000900033010008A1010008330100083301000802
:1000A0003301000833010008330100083301000860
:1000B0003301000833010008330100083301000850
:1000C0003301000833010008330100083301000840
:1000D0003301000871030008090400083301000817
:1000E000330100083301000833010008000000005C
:1000F0000000000000000000000000000000000000
:1001000033010008DFF80CD000F038F80048004751
:100110009D0D0008B036002006488047064800477D
:10012000FEE7FEE7FEE7FEE7FEE7FEE7FEE7FEE7A7
:10013000FEE7FEE70D0300080501000840EA0103A1
:100140009B0703D009E008C9121F08C0042AFAD28D
:1001500003E011F8013B00F8013B521EF9D2704751
:1001600010B5002200E0521C835C8C5CA34201D1DC
:10017000002BF8D1D8B2E1B2401A10BD064C074DA1
:1001800006E0E06840F0010394E807009847103467
:10019000AC42F6D3FFF7BAFF641D0008841D0008C7
:1001A00010B5012001F094F90348006840F02000E8
:1001B0000149086010BD00001064004028B1012210
:1001C000044B1A701A46518002E0024A0023136061
:1001D00070470000DC00002028B10122044B1A7097
:1001E0001A46518002E0024A002313607047000063
:1001F000D000002010B5002807DA0A07140E054ABF
:1002000000F00F031B1FD45403E00A07130E024A29
:10021000135410BD18ED00E000E400E070B5054691
:100220000C4615B10CB1802C01D9002070BD2246BE
:1002300029460748FFF782FF002006490880064844
:10024000046040F20631054801F03BFD0120EDE776
:10025000AF140020C8000020CC0000200044004063
:1002600070B505460C4615B10CB1802C01D90020A3
:1002700070BD224629460A48FFF760FF0020094961
:1002800008800948046040F20631084801F019FD71
:1002900040F20631054801F021FD0120E8E70000A9
:1002A000AF150020D4000020D80000200038014005
:1002B00013480068401C1249086000BF11480078CC
:1002C000D8B110484088401C0E49488008464088F4
:1002D000042808DB002048800B48006840F08000BC
:1002E0000949086009E007484088022805D1064806
:1002F000006840F040000449086000BF70470000FB
:10030000940000200C0000201000002010B51448BC
:10031000006840F001001249086008464068114931
:1003200008400F494860084600680F4908400C49DA
:1003300008600846006820F480200860084640688D
:100340000A490840064948600846006806490840CE
:10035000034908604FF41F00886001F0E3FB10BD03
:10036000001002400C00FFE8FFFFF6FEFFFF00F761
:1003700010B505211E4801F078FC012818D11C4851
:1003800001F01CFCC4B21B480088802800D310BDBB
:1003900000210846FFF712FF164801880088401C1C
:1003A000144A10801448445405210120FFF706FF29
:1003B00006210F4801F059FC012816D10F4800888A
:1003C0000F490968884205D340F20631084801F018
:1003D0006BFCDCE7094802880088401C074B18804A
:1003E0000848815C024801F0EEFB00BFCFE7000047
:1003F00000380140D60000202F160020D400002035
:10040000D8000020AF15002010B505211E4801F0CE
:100410002CFC012818D11C4801F0D0FBC4B21B48A9
:100420000088802800D310BD00210846FFF7D4FEC5
:10043000164801880088401C144A1080144844540F
:1004400005210120FFF7C8FE06210F4801F00DFC31
:10045000012816D10F4800880F490968884205D342
:1004600040F20631084801F01FFCDCE70948028829
:100470000088401C074B18800848815C024801F046
:10048000A2FB00BFCFE7000000440040CA000020EC
:100490002F150020C8000020CC000020AF14002041
:1004A00010B540F2026000F01BFE4FF4C06000F097
:1004B00017FE40F20E6000F013FE4FF400730322AB
:1004C00018211D4800F0CCFB4FF480630322042167
:1004D000194800F0C5FB194801F07AFB4FF41641AA
:1004E000164801F023FB0021144801F033FC0021E1
:1004F000124801F01FFC0021104801F00BFC002104
:100500000E4801F0C9FB00210C4801F0BDFB04219D
:100510000A4801F007FC0821084801F013FC4FF4D9
:10052000407000F037FD00220121252000F0DCFCA6
:10053000024801F095FB10BD000801400038014061
:1005400010B540F2026000F0CBFD4FF4C06000F047
:10055000C7FD0423032218211E4800F081FB082355
:10056000032204211B4800F07BFB40F2117000F0D5
:10057000B7FD194801F02CFB4FF41641164801F065
:10058000D5FA0021144801F0E5FB0021124801F0E2
:10059000D1FB0021104801F0BDFB00210E4801F005
:1005A0007BFB00210C4801F06FFB04210A4801F09D
:1005B000B9FB0821084801F0C5FB4FF4407000F07A
:1005C000E9FC00220121262000F08EFC024801F007
:1005D00047FB10BD000801400044004002E008C88D
:1005E000121F08C1002AFAD170477047002001E0AD
:1005F00001C1121F002AFBD1704730B5034688188D
:100600009C8890FBF4F504FB150080B230BD38B532
:10061000044601226946204600F031F8002802DD38
:100620009DF8000038BDFF20FCE770B504460E467B
:1006300015462660A580204600F001F870BD10B573
:1006400003680279002102E059544C1CE1B2914246
:10065000FADB541E04810024C48010BD13B5044687
:10066000012201A9204600F032F81CBD70B50446F5
:100670000D46E1882A462046FFF7BFFF70BD2DE9F1
:10068000F04105460C461646274604EB060811E0E5
:10069000E8882989884203D1E01B80B2BDE8F08157
:1006A000E9882868405C207001212846FFF7DEFFBA
:1006B000E880641C4445EBD33046EFE770B5044650
:1006C0000D4621892A462046FFF797FF70BD2DE988
:1006D000F04705460C461646274604EB060912E08D
:1006E00001212846FFF7EAFF8046E888404503D10C
:1006F000E01B80B2BDE8F08720782A8929688854F9
:10070000A5F80880641C4C45EAD33046F2E713B5DF
:100710000446012201A92046FFF7D9FF1CBD0000B5
:1007200010B504460548844207D140F2194000F054
:10073000F7FC40F2194000F0E3FC10BD00640040FB
:1007400010B50021837A012202FA03F13E4A1268B1
:1007500042F001023C4B1A603B4A1C3212688A4349
:10076000394B1C331A60C289DAB9374A0C32126825
:100770008A43354B0C331A60C288344B03EA024279
:1007800043881A434389304C403444F833208288EC
:100790002E4B03EA024203881A43438904EBC30346
:1007A0005A60C289012A1BD1274A0C3212680A43B7
:1007B000254B0C331A600288244B03EA024243881B
:1007C0001A434389204C403444F8332082881F4B1D
:1007D00003EA0242C3881A43438904EBC3035A6005
:1007E00082893AB9184A121D12688A43164B1B1D9A
:1007F0001A6006E0144A121D12680A43124B1B1DB0
:100800001A6002893AB9104A143212688A430E4BB0
:1008100014331A6006E00C4A143212680A430A4B79
:1008200014331A60027C012A06D1074A1C3212686E
:100830000A43054B1C331A60034A126822F0010276
:10084000014B1A6010BD0000006600400000FFFF71
:1008500070B502464FF6FF730020146824F00204BE
:100860001460146844F00104146000E05B1E5468D6
:1008700004F001040CB9002BF8D1546804F0010411
:100880000CB9002074E00C784FF0404505EA847400
:100890004D784FF0407606EA05652C438D784FF48D
:1008A000702606EA05452C43CD784FF4E00606EAAB
:1008B00005552C434D896D1EC5F309052C43D461A4
:1008C0000C79012C04D1146844F08004146003E016
:1008D000146824F0800414604C79012C04D114684D
:1008E00044F04004146003E0146824F040041460F1
:1008F0008C79012C04D1146844F02004146003E0C6
:10090000146824F020041460CC79012C04D11468FC
:1009100044F01004146003E0146824F01004146020
:100920000C7A012C04D1146844F00804146003E02C
:10093000146824F0080414604C7A012C04D1146863
:1009400044F00404146003E0146824F00404146008
:10095000146824F0010414604FF6FF7300E05B1E7E
:10096000546804F001040CB1002BF8D103B101204C
:1009700070BD42690A434261704700B503460122D7
:1009800000BF00F00BF802465B1E012A01D1002BCC
:10099000F7D1012A00D10422104600BD00200A49E7
:1009A000C96801F0010109B101200CE00649C968DC
:1009B00001F0100109B1032005E00349C96801F005
:1009C000040101B1022070470020024000B5034637
:1009D000012200BF00F00CF802465B1E012A01D183
:1009E000002BF7D1012A00D10422104600BD0000DF
:1009F00000200A49C96C01F0010109B101200CE095
:100A00000649C96C01F0100109B1032005E0034952
:100A1000C96C01F0040101B10220704700200240BE
:100A2000064A02EB9011096800F01F0301229A4068
:100A30001143024B03EB90121160704700200240FB
:100A40000848006940F080000649086106480088AF
:100A5000B0F5007F04D90846006D40F080000865BD
:100A60007047000000200240E0F7FF1F30B5054648
:100A700036480088B0F5007F48D9354885421ED2F7
:100A80004FF47020FFF779FF0446002C5BD131480A
:100A9000006940F002002F4908610846456100697D
:100AA00040F0400008614FF47020FFF766FF0446F5
:100AB0002848006920F002002649086143E04FF40D
:100AC0007020FFF783FF0446002C3CD12148006DC5
:100AD00040F002001F49086508464565C06900F0FE
:100AE000020008B1084645611A48006D40F0400018
:100AF000184908654FF47020FFF768FF0446154851
:100B0000006D20F00200134908651CE04FF47020CE
:100B1000FFF733FF0446B4B90E48006940F0020005
:100B20000C49086108464561006940F040000861D1
:100B30004FF47020FFF721FF04460648006920F0BB
:100B4000020004490861204630BD0000E0F7FF1FA5
:100B5000FFFF0708002002400C48006900F08000F9
:100B600020B10B48094948600A4848600A48008893
:100B7000B0F5007F09D90548006D00F0800020B174
:100B80000348024948640348486470470020024013
:100B900023016745AB89EFCDE0F7FF1F70B5044631
:100BA0000D4600262A480088B0F5007F35D929482F
:100BB000844219D24FF47020FFF7DFFE0646002E64
:100BC00043D12548006940F00100234908612560B0
:100BD0004FF47020FFF7D1FE06461F48006920F051
:100BE00001001D49086130E04FF47020FFF7EEFE70
:100BF000064656BB1848006D40F0010016490865CE
:100C000025604FF47020FFF7E1FE06461248006DA4
:100C100020F001001049086517E04FF47020FFF73D
:100C2000ACFE06468EB90C48006940F001000A4946
:100C3000086125604FF47020FFF79FFE06460648C6
:100C4000006920F0010004490861304670BD0000D1
:100C5000E0F7FF1FFFFF07080020024041617047D7
:100C6000F0B5044616460025002201F00F0501F0FC
:100C7000100707B1354300201EE0012787401F40C1
:100C8000C7B122684FEA800C0F2707FA0CF7BA4366
:100C9000870005FA07F73A43282904D1012787403E
:100CA0001F40676105E0482903D1012787401F40A5
:100CB00027612260471CB8B20828DED3082022E052
:100CC000012787401F40E7B16268A0F108074FEA9B
:100CD000870C0F2707FA0CF7BA43A0F10807BF00EB
:100CE00005FA07F73A43282904D1012787401F4016
:100CF000676105E0482903D1012787401F4027612C
:100D00006260471CB8B21028DAD3F0BDF0B50A46CD
:100D1000002300240021002500F00046B6F1004F1A
:100D200002D11D4EF16901E01B4E7168C0F303450D
:100D300083B200F44016B6F5401F08D121F070616F
:100D4000154E766826F07066134F7E6012E000F450
:100D50008016B6F5801F06D1032606FA05F4A143D6
:100D600041F0706106E0460D360103FA06F6B14324
:100D700041F0706122B1460D360103FA06F63143A7
:100D800000F00046B6F1004F02D1034EF16101E0E0
:100D9000014E7160F0BD00000000014008B545A0A3
:100DA00000680090012000F01BFD00BF4248006871
:100DB0000A21B0FBF1F4601EB0F1807F00D30FE098
:100DC000601E4FF0E02148610F214FF0FF30FFF728
:100DD00011FA00204FF0E02188610720086100BF70
:100DE0000021481EFFF706FA00BF00BFFFF758FBBF
:100DF000FFF7A6FB0120314908700420488040F22B
:100E0000026000F06DF94FF48053032210212C484A
:100E1000FFF726FF4FF480512948FFF71FFF40F2EC
:100E2000026000F05DF98023032210212448FFF7BF
:100E300017FF80212248FFF711FF00BF00F080F963
:100E4000032269467F2000F0ADFB31E000F020FA7C
:100E50001C480068B0F5167F0AD9002000F0C0FCDD
:100E6000002018490860032269467F2000F09AFBA1
:100E70001548007800F0400050B100BF13480178D9
:100E8000FFF7EEF91048006820F040000E490860B6
:100E90000D48007800F0800050B100BF0B48017889
:100EA000FFF7BCF90848006820F080000649086098
:100EB000CCE70000F0420000000000200C00002001
:100EC00000080140940000201000002014000020C1
:100ED00000F01F0201219140024A431142F8231001
:100EE0007047000080E100E02DE9F04103460D4627
:100EF000164600240027A0462448006800F4E0605D
:100F0000B0F5A06F15D006DCB0F5407F18D0B0F575
:100F1000806F19D110E0B0F5C06F06D0B0F5E06F6A
:100F200012D100274FF0040815E001274FF0030805
:100F300011E00227B8460EE003274FF001080AE04F
:100F400004274FF0000806E04FF4A06000F022F8FC
:100F50000227B84600BF00BFC7F1040005FA00F43D
:100F6000C8F104010F20C840304004432401084860
:100F7000C45403F01F01012088405911890001F178
:100F8000E021C1F80001BDE8F08100000CED00E0B7
:100F900000E400E002490143024A1160704700008A
:100FA0000000FA050CED00E0024A0A400243024B41
:100FB0001A60704780FFFF1F08ED00E02DE9F04F39
:100FC0008BB00746002009903EA090E8004CC06816
:100FD000CDE905BECDF810A007900FF2EC0ADAE9D2
:100FE000000ACDE9020A0FF2E00ADAE9000ACDE9C7
:100FF000000A38484068C0F381000A900A9820B17E
:10100000012804D0022829D103E0334928E03249DD
:1010100026E03048406800F48038B8F5803F09D1B8
:101020002D4C2C48406800F40039B9F5003F02D13E
:10103000641000E0294C27484068C0F383422548EB
:10104000406800F0006008B142F010020F2A01D29F
:10105000921C00E0521C04FB02F101E01E4900BF9B
:1010600000BF1C484068C0F3031504A8465D21FA80
:1010700006F318484068C0F3022502A8465D23FA2B
:1010800006FC14484068C0F3C2251DF8056023FA29
:1010900006F0089037B1012F06D0022F06D0032F9B
:1010A0000AD106E0099108E0099306E0CDF824C0D2
:1010B00003E00898099000E000BF00BF09980BB05A
:1010C000BDE8F08F000000000000000001020304F2
:1010D000060708090010024000127A0000093D00CE
:1010E000064A02EB9011096800F01F0301229A40A2
:1010F0001143024B03EB9012116070470010024045
:10110000064A02EB9011096800F01F0301229A4081
:101110009143024B03EB90121160704700100240A4
:10112000064A02EB9011096800F01F0301229A4061
:101130001143024B03EB9012116070470010024004
:1011400000B589B000BF06223B493C48FFF76DFA65
:101150000B223B493B48FFF768FA40F20360FFF778
:10116000BFFF4FF4C060FFF7BBFF40F21970FFF7FD
:10117000B7FF00BF00BF4FF48073032248213248FD
:10118000FFF76EFD4FF40073032218212E48FFF77E
:1011900067FD01214FF4EA10FFF7B8FD00BF2B48AF
:1011A000FFF7BEFA00208DF81C008DF81D008DF8A9
:1011B0001E008DF81F008DF8200001208DF8210001
:1011C00000208DF8190004208DF81A0002208DF8F7
:1011D0001B0000208DF818001820ADF8220006A989
:1011E0001A48FFF735FB0020ADF80E00ADF81000EF
:1011F0000120ADF812000020ADF804004FF4057096
:10120000ADF806000020ADF808004FF47F70ADF88F
:101210000A000120ADF80C008DF8140001A8FFF7BA
:101220008FFA002211461520FFF75EFE10210748B5
:10123000FFF79FFB09B000BD9D0000208014002037
:101240008C14002098140020000C01400064004021
:1012500010B51520FFF73CFE0148FFF761FA10BDFD
:10126000006400400948016801F0806008B1002076
:10127000704701F0006008B10120F9E701F08050EB
:1012800008B10220F4E70320F2E700000864004000
:1012900038B500F001FA12E09DF8000000EB4010B4
:1012A0000B4901EBC004E288607804F1080100F00A
:1012B00015F800BF9DF800100648FFF7CFF901228E
:1012C00069460548FFF7DBF90028E5DC38BD00007A
:1012D000080A002098140020B80000202DE9F74FDC
:1012E00082B089461446022C02DA05B0BDE8F08FC0
:1012F000B9F800A04FF6F0700AEA000044F2F021BD
:10130000884200D0F1E700203C49086009F102065C
:10131000A01E84B2AAF58440F038062859D2DFE82E
:1013200000F003050E292E52002555E000BF0020D5
:101330003349086000F042FB002500BF4CE037460F
:10134000A046B8F1070F02DA4FF0FF3010E0384640
:1013500000F023FA8346F81C00F028FA0190584662
:10136000019900F039FB08B1002001E04FF0FF3097
:10137000054631E02146304600F0ECFAB5E7B046CC
:101380002746032F02DA4FF0FF301AE0404600F004
:1013900004FA83461A48006858450BD1F81E87B2F4
:1013A000394608F1030000F0D5FA154800683844C2
:1013B000134908601248016808F1010000F006FABC
:1013C0000320054608E0002000F00AFA4FF0FF3540
:1013D00002E04FF0FF3500BF00BF002D03DA00250B
:1013E0000120307001E000203070E81C82B24946D4
:1013F000029800F045F900BF77E700009400002054
:10140000C40000202DE9F0410546002609E01849F6
:1014100051F826004178A94201D1BDE8F081701C45
:10142000C6B2144800788642F1DB124800780A28D8
:101430001BD21148FFF7EBF80746FF2F01D1002020
:10144000EBE707EB47100D4901EBC0046570FF2087
:10145000E07007480749097840F8214005480078BE
:10146000401C044908702046D7E70020D5E700005B
:10147000581400209C00002098140020080A002026
:10148000024600211AE0104850F82100904213D182
:101490000E480078401E0D4B187007E00A4B481CA0
:1014A00053F8200043F82100481CC1B207480078D7
:1014B0008142F3DB01207047481CC1B20348007829
:1014C0008142E0DB0020F6E7581400209C00002059
:1014D0002DE9F05F0646304901EB0610D0F8B095D3
:1014E00009F00600042802D00120BDE8F09F4FEA71
:1014F000D905294901EB0610D0F8B495C5F3C610FB
:10150000FFF780FF04460CB90020EEE7C5F38437EF
:10151000C5F3C44AE078B8420ED0012F01D00120B3
:10152000E3E7C5F30160A07005F07F0020700020A4
:10153000A0800220E07003E0781C00F01F00E07043
:10154000A18804F1080001EB0008A08809F00F0150
:101550000844A080104901EB0610D0F8B805C8F87F
:10156000000001EB0610D0F8BC05C8F80400BA452D
:1015700010D1A088E0800948201A4FF4847190FBB4
:10158000F1F000F0FF0B59460548FFF7C0F8204680
:10159000FFF776FF0120A8E700600040080A00205E
:1015A000B8000020F8B506460C4615462346012231
:1015B00042213046009500F031F8F8BD70B5164D67
:1015C00005EB0014D4F8844524F00F042E4606EBF6
:1015D0000015C5F88445354605EB0014D4F884455C
:1015E0001C4306EB0015C5F8844506EB001514688E
:1015F000C5F88845042B04DD06EB00155468C5F8D2
:101600008C456FF0070404EAC104641D024E06EB2A
:101610000015C5F8804570BD006000402DE9F04719
:1016200006460F4690469946DDF820A01148FEF781
:10163000EEFF0546FF2D02D10020BDE8F08705EB47
:1016400045100D4901EBC0040020A08084F8028001
:1016500026706770A4F806A05246494604F10800B7
:10166000FEF76CFD29460548FFF751F800F014F825
:101670000120E2E780140020E0040020AC000020FC
:10168000F8B506460C46154623460222422130464E
:101690000095FFF7C3FFF8BD38B532E01A4800687F
:1016A000C8B119480068808817490968C988884204
:1016B00004DA1548006800F02FF823E012480068AB
:1016C0001249401A4FF4847190FBF1F0C4B22146E4
:1016D0000F48FEF7C3FF012269460E48FEF7CFFF11
:1016E000002809DD9DF8000000EB4010074901EBE0
:1016F000C0000549086003E000200349086001E0DC
:1017000000BFCBE700BF38BD98000020E0040020F8
:1017100080140020AC0000202DE9F0430446FFF7C0
:10172000A1FD8046B8F1030F02D10020BDE8F0838F
:10173000E188C81DC11700EB5171C1F3C706A0882D
:10174000C11700EB5171C910491CCFB2A0784FF0FE
:10175000C05141EA006006F01F0140EAC14007F0B5
:101760001F0140EA813021780843617840EAC119BD
:10177000E088A188401A85B2082D00DD0825EBB26B
:10178000A18804F108000A1849464046FFF716FFF1
:10179000A0882844A0800120C8E7014608784A783C
:1017A00040EA02208A7840EA024070470146087801
:1017B0004A7840EA02208A7840EA0240CA7840EA41
:1017C0000260704701700A124270704710B50446FB
:1017D0000B4699B22046FFF7F5FF180CA07010BD1C
:1017E000F8B505462B4C2C4EA068401C88B92B48F8
:1017F000009000230422694604F1080000F00EF96D
:1018000000F09EF8074601230C22214600F006F95D
:1018100000BF23A13046FEF7A3FC08B10020F8BDAD
:1018200000F08EF804462DB11C49A068884214D0FF
:101830000020F4E700F038F8A0F500502168884255
:1018400001D20020EBE713481030216800F034F893
:101850006168884201D00020E1E72520FFF738FBCE
:101860002620FFF735FBFFF7F3FC00204FF0E021C7
:10187000086108491031086880F3088800BF00211A
:1018800004481030FFF790FB024910314868804748
:101890000020C4E7F01F000800280008443322118C
:1018A00050533130300000000248006800048009C5
:1018B00070470000E0F7FF1FF0B503460C464FF0FD
:1018C000FF311A46161912E0107800250CE081EA63
:1018D000000707F001071FB1074F87EA510100E039
:1018E000490840106F1CFDB2082DF0DB521CB242BB
:1018F000EAD3C843F0BD00002083B8ED10B540F234
:101900000730FFF78DF810BD10B50446A2B20123D1
:1019100008490948006800F081F808B9002010BDA6
:1019200005480068204404490860002003490880F5
:101930000120F4E7E000002004000020080000205F
:1019400010B5FFF7B1FF0446A4F5806000F1006018
:1019500010BD000070B506460C4627E0154800880B
:10196000C0F5806085B2AC420DDA1349114A128885
:10197000881822463146FEF7E1FB0E4800882044D5
:101980000C49088013E00C490A4A128888182A4634
:101990003146FEF7D3FB4FF48060FFF7B5FF08B97F
:1019A000002070BD2E44601B84B200BFD6E700BF8C
:1019B0000120F6E708000020E00000200348044969
:1019C00008600020034908807047000000200008DC
:1019D00004000020080000207CB504460D460D4898
:1019E0000088FFF791FF08B900207CBD21460A4816
:1019F000FFF762FFA84201D00020F6E700940195AE
:101A0000FFF79EFF064601230822694600F006F80C
:101A1000EBE7000008000020002000082DE9F04757
:101A200006460D4617469846FFF796F8B8F1000FA0
:101A300008D0FFF763FF3046FFF718F810B1002019
:101A4000BDE8F0872C46F81CC11700EB9171891096
:101A500004EB81090AE0FFF751FF30462168FFF7E8
:101A60009DF808B10020EBE7241D361D4C45F2D34C
:101A7000FEF7E6FF0120E3E700200021264A126876
:101A800042F00102244B1A6000BF401C224A126837
:101A900002F0020111B9B0F5A06FF6D11E4A12682A
:101AA00002F002020AB900BFFEE71B4A52681A4B55
:101AB0005A601A4652685A601A46526842F4806266
:101AC0005A601A465268154B1A40134B5A601A4610
:101AD0005268134B1A43104B5A601A46126842F070
:101AE00080721A6000BF0C4A126802F00072002A6D
:101AF000F9D0094A526822F00302074B5A601A468D
:101B0000526842F002025A6000BF034A526802F073
:101B10000802002AF9D0704700100240FFFFC3F707
:101B20000000280810B5FFF7A7FF10BD2DE9F0470A
:101B300004460D460027B846B94600261D49601ADE
:101B40008C421CD006DC1C48204470B1B0F5806F7C
:101B50001FD10FE0B0F5806F16D0B0F56C4F18D1E3
:101B60000320FFF72BFA074614E00220FFF726FABE
:101B700007460FE00220FFF721FA07460AE002209D
:101B8000FFF71CFA074605E00220FFF717FA0746A1
:101B900000E000BF00BF07EB5500B0FBF5F64FF6C5
:101BA000F07006EA000806F00F0948EA0900A06094
:101BB000BDE8F087004C004000BCFFBF014648680C
:101BC000C0F308007047C1F308024260704700008C
:101BD00010B504462049601A8C4228D006DC1F4804
:101BE000204490B1B0F5806F33D117E0B0F5806F2D
:101BF00026D0B0F56C4F2CD140F20E30FFF790FAA2
:101C000040F20E30FFF77CFA24E040F21140FFF77B
:101C100087FA40F21140FFF773FA1BE040F21240DE
:101C2000FFF77EFA40F21240FFF76AFA12E040F244
:101C30001340FFF775FA40F21340FFF761FA09E02D
:101C400040F21440FFF76CFA40F21440FFF758FAE4
:101C500000E000BF00BF10BD004C004000BCFFBF53
:101C6000C16841F40051C160704710B5024602EBF3
:101C70009110006801F01F040123A340184008B12F
:101C8000012010BD0020FCE70A460021416921F433
:101C900000711143416170470A460021416921F4F6
:101CA000807111434161704710B5C1F389128258A8
:101CB00001F01F040123A3409A43C1F38913C250CA
:101CC00010BD10B5C1F38912825801F01F04012321
:101CD000A3401A43C1F38913C25010BD70B5024628
:101CE00000230024C1F38910105801F01F060125BC
:101CF000B54000EA050302EB91500068C1F30446C9
:101D00000125B54000EA050414B10BB1012070BDF6
:101D10000020FCE7C26822F4C062C260C2680A43C5
:101D2000C26070470A460021C16821F004011143D6
:101D3000C1607047026922F44052026102690A439D
:101D4000026170470A460021C16821F00801114371
:101D5000C1607047C26822F48052C260C2680A4300
:101D6000C2607047841D000800000020E0000000F1
:101D7000DC050008641E0008E0000020D0350000EB
:101D8000EC05000800F36F060000000000000000F2
:101D90000000000000000000173142108BBE16004A
:101DA000000000000000050000000000000000002E
:101DB0000000000000000000000000000000000023
:101DC0000000000000000000000000000000000013
:101DD0000000000000000000000000000000000003
:101DE00000000000000000000000000000000000F3
:101DF00000000000000000000000000000000000E3
:101E000000000000000000000000000000000000D2
:101E100000000000000000000000000000000000C2
:101E200000000000000000000000000000000000B2
:101E3000A30000200600000000000000A414002001
:101E40000B00000000000000000000000000000087
:101E50000000000000000000000000000000000082
:041E6000000000007E
:0400000508000105E9
:00000001FF
